:100000000C9444000C946C000C946C000C946C00E8
:100010000C946C000C946C000C946C000C946C00B0
:100020000C946C000C946C000C946C000C946E009E
:100030000C946C000C946C000C946C000C946C0090
:100040000C946C000C946C000C9460030C946C0089
:100050000C946C000C946C000C946C000C946C0070
:100060000C946C000C946C0005A84CCDB2D44EB925
:100070003836A9020C50B9918688083CA6AAAA2A4B
:10008000BE000000803F3E0111241FBECFEFD8E02C
:10009000DEBFCDBF11E0A0E0B1E0E4E3F4E102C0D7
:1000A00005900D92A232B107D9F713E0A2E2B1E0B8
:1000B00001C01D92AC3AB107E1F710E0C8E8D0E00A
:1000C00004C02297FE010E947F08C638D107C9F7F5
:1000D0000E9402010C94180A0C9400001F920F92C7
:1000E0000FB60F9211242F933F934F935F936F930B
:1000F0007F938F939F93AF93BF93CF93DF93EF93B0
:10010000FF9385B190E2892785B9C0E0D0E0E09106
:100110002403F0912503EE5DFE4F86E293E06081BB
:100120000E9445018091240390912503019660E08F
:1001300072E00E94E20790932503809324032196A6
:1001400081E0C034D80719F786E293E060E00E94AE
:100150004501FF91EF91DF91CF91BF91AF919F91B9
:100160008F917F916F915F914F913F912F910F9060
:100170000FBE0F901F901895AF92BF92CF92DF9253
:10018000EF92FF920F931F93CF93DF93C2E2D1E0E0
:100190000F2EF0E0AF2EF0E0BF2EF0E0CF2EF0E01B
:1001A000DF2EF02DC601B5010E9483087B018C0172
:1001B000C601B50128ED3FE049E45CE30E941A0561
:1001C0005B016C01C801B70120E030E04EEF52E462
:1001D0000E94470520E030E040E053E40E941A0509
:1001E0000E944106699383E0C232D807D9F6DF91B5
:1001F000CF911F910F91FF90EF90DF90CF90BF9024
:10020000AF9008951F930E94BC0086E293E040E007
:1002100052EC61E070E00E945201259A80E285B9BB
:100220008091810088608093810080916F0082605E
:1002300080936F0086E891E0909389008093880016
:10024000789410E286E293E00E944F011816190696
:10025000CCF785B1812785B986E293E00E944C01F5
:10026000813681F786E293E060E071E00E94A601AA
:1002700080918100856080938100E4CF87E191E0E7
:1002800090932703809326030895862F0E941F03CF
:1002900008950E94570308950E94380308950E940C
:1002A00027030895CB01BA010E94E6020895DC01FC
:1002B000ED91FC910190F081E02D09950895DC010C
:1002C000ED91FC910190F081E02D099508950F9337
:1002D0001F93CF93DF938C01EB0109C02196D801C6
:1002E000ED91FC910190F081E02DC80109956881A4
:1002F0006623A1F7DF91CF911F910F9108950F937E
:100300001F938C01DC01ED91FC910190F081E02DB7
:100310006DE00995D801ED91FC910190F081E02DFF
:100320006AE0C80109951F910F9108950F931F93DB
:100330008C01DC01ED91FC910190F081E02D09959B
:10034000C8010E947F011F910F9108950F931F9381
:100350008C010E946701C8010E947F011F910F91CB
:1003600008950F931F938C01DC01ED91FC91019096
:10037000F081E02D0995C8010E947F011F910F9126
:1003800008952F923F924F925F926F927F928F9239
:100390009F92AF92BF92CF92DF92EF92FF920F9314
:1003A0001F93DF93CF93CDB7DEB7A0970FB6F89426
:1003B000DEBF0FBECDBF1C016A017B014115510597
:1003C0006105710549F4DC01ED91FC910190F0812A
:1003D000E02D60E3099554C0882499245401422EED
:1003E00055246624772401E010E00C0F1D1F080D32
:1003F000191DC701B601A30192010E94F507F8017A
:1004000060830894811C911CA11CB11CC701B6011A
:10041000A30192010E94F507C901DA016C017D0177
:10042000C114D104E104F104F1F681E0E82EF12CCD
:10043000EC0EFD1EE80CF91C3E010894611C711CB9
:10044000D501C4010197A109B1096C01C818D908E7
:1004500014C0F601EE0DFF1D60816A3010F4605D7E
:1004600001C0695CD101ED91FC910190F081E02D1A
:10047000C10109950894E108F1086E147F0449F759
:10048000A0960FB6F894DEBF0FBECDBFCF91DF911F
:100490001F910F91FF90EF90DF90CF90BF90AF90A2
:1004A0009F908F907F906F905F904F903F902F9094
:1004B00008952AE00E94C10108950F931F938C01B3
:1004C0000E945902C8010E947F011F910F91089557
:1004D000AB0160E070E00E94590208950F931F93F2
:1004E0008C01AB0160E070E00E945902C8010E94DB
:1004F0007F011F910F910895EF92FF920F931F9329
:10050000CF93DF93EC017A018B0177FF0FC0E88175
:10051000F9810190F081E02D6DE20995109500952B
:10052000F094E094E11CF11C011D111D2AE0B801BA
:10053000A701CE010E94C101DF91CF911F910F91C0
:10054000FF90EF9008950F931F938C010E947C02FF
:10055000C8010E947F011F910F910895AB0166278A
:1005600057FD6095762F0E947C0208950F931F938C
:100570008C01AB01662757FD6095762F0E947C02A7
:10058000C8010E947F011F910F910895DC01211580
:10059000310541F4ED91FC910190F081E02D642F43
:1005A000099508952A30310519F40E947C020895B6
:1005B0000E94C10108950F931F938C010E94C602EF
:1005C000C8010E947F011F910F910895EF92FF9241
:1005D0000F931F937B018C0122E030E040E050E05C
:1005E0000E941708205C3D4B404F5F4FCA01B90184
:1005F000A80197010E941708C901DA010197A10912
:10060000B109292F3A2F4B2F552747FD5A950196AF
:10061000A11DB11D2093C50081508093C400E1EC61
:10062000F0E0808180618083808188608083808128
:10063000806880831F910F91FF90EF900895982F0D
:100640008091C00085FFFCCF9093C60008958091F3
:1006500028039091290380589F4F20912A033091BD
:100660002B03821B930B60E870E00E94E207089561
:1006700040912A0350912B038091280390912903E4
:100680008417950719F42FEF3FEF0FC0FA01E45DCF
:10069000FC4F2081CA01019660E870E00E94E207E9
:1006A00090932B0380932A0330E0C9010895809131
:1006B0002A0390912B039093290380932803089594
:1006C0001F920F920FB60F9211242F933F934F93C7
:1006D0005F936F937F938F939F93AF93BF93EF93AA
:1006E000FF934091C600E0912803F0912903CF01C8
:1006F000019660E870E00E94E2079C0180912A0365
:1007000090912B032817390739F0E45DFC4F4083A3
:100710003093290320932803FF91EF91BF91AF916C
:100720009F918F917F916F915F914F913F912F9109
:100730000F900FBE0F901F901895A0E0B0E0E3EA75
:10074000F3E00C944608DC012B01FA019C919230F5
:1007500008F439C1EB018881823008F433C1943048
:1007600069F4843009F02FC111969C911197898109
:10077000981709F428C1A9E1B1E025C1843009F432
:1007800021C18230A9F4923009F01DC19A01AD0156
:1007900088E0EA010990AE01E90109929E018150C9
:1007A000C1F7E201898111969C918923818308C157
:1007B000923009F407C112962D903C901397EB01EB
:1007C0008A819B811496AD90BD90CD90DC90179757
:1007D000EC80FD800E811F819101281B390BB9012E
:1007E00037FF04C066277727621B730B60327105E1
:1007F0000CF061C0121613066CF537014801062E85
:1008000004C096948794779467940A94D2F721E071
:1008100030E040E050E004C0220F331F441F551F5A
:100820006A95D2F721503040404050402E213F2160
:1008300040235123211531054105510521F021E0C7
:1008400030E040E050E079018A01E628F7280829E5
:1008500019293CC0232BD1F1260E371E3501460144
:10086000062E04C096948794779467940A94D2F7DE
:1008700021E030E040E050E004C0220F331F441F6D
:10088000551F6A95D2F721503040404050402A21F0
:100890003B214C215D21211531054105510521F0F8
:1008A00021E030E040E050E059016A01A628B72875
:1008B000C828D9280BC0821593052CF01C01AA2446
:1008C000BB24650103C0EE24FF24870111969C918F
:1008D000D20111968C91981709F445C0992339F0EB
:1008E000A80197012A193B094C095D0906C0A60118
:1008F00095012E193F09400B510B57FD08C011827D
:100900003382228224833583468357831DC081E04E
:1009100081833382228288279927DC01821B930BF3
:10092000A40BB50B84839583A683B7830DC0220FD8
:10093000331F441F551F2483358346835783828189
:1009400093810197938382832481358146815781E6
:10095000DA01C9010197A109B1098F5F9F4FAF4F1C
:10096000BF4328F30BC0918333822282EA0CFB1C25
:100970000C1D1D1DE482F5820683178383E08083AE
:10098000248135814681578157FF1AC0C901AA27A2
:1009900097FDA095BA2F81709070A070B070569599
:1009A000479537952795822B932BA42BB52B8483C2
:1009B0009583A683B78382819381019693838283F3
:1009C000DF0101C0D201CD01CDB7DEB7E2E10C9469
:1009D0006208A0E2B0E0EFEEF4E00C945208698304
:1009E0007A838B839C832D833E834F835887E9E0F2
:1009F000EE2EF12CEC0EFD1ECE010196B7010E94E9
:100A00006A078E010F5E1F4FCE010596B8010E9446
:100A10006A078A8991E089278A8BC701B801AE01EC
:100A2000475E5F4F0E949D030E949506A096E6E0F8
:100A30000C946E08A0E2B0E0E0E2F5E00C945208FD
:100A400069837A838B839C832D833E834F8358876E
:100A5000F9E0EF2EF12CEC0EFD1ECE010196B70150
:100A60000E946A078E010F5E1F4FCE010596B801E6
:100A70000E946A07C701B801AE01475E5F4F0E943E
:100A80009D030E949506A096E6E00C946E08A0E2F5
:100A9000B0E0EDE4F5E00C94460869837A838B833B
:100AA0009C832D833E834F835887CE010196BE01E0
:100AB000675F7F4F0E946A07CE010596BE016F5E99
:100AC0007F4F0E946A079985923088F08989823029
:100AD000C8F0943019F4823051F404C0843029F401
:100AE000923081F489E191E0C6C0923049F420E06F
:100AF0009A858A89981321E02A87CE010996BBC07E
:100B0000823049F420E09A858A89981321E02A8B63
:100B1000CE014196B0C02D843E844F8458886D88A4
:100B20007E888F88988CEE24FF248701AA24BB241A
:100B3000650140E050E060E070E0E0E0F0E0C1011D
:100B400081709070892BE9F0E60CF71C081D191DC7
:100B50009A01AB012A0D3B1D4C1D5D1D80E090E00C
:100B6000A0E0B0E0E614F7040805190520F481E0E0
:100B700090E0A0E0B0E0BA01A901480F591F6A1F38
:100B80007B1FAA0CBB1CCC1CDD1C97FE08C081E09F
:100B900090E0A0E0B0E0A82AB92ACA2ADB2A319660
:100BA000E032F10549F0660C771C881C991C5694BC
:100BB000479437942794C3CFFA85EA892B893C89D7
:100BC0008B859C85280F391F2E5F3F4F17C0CA01A8
:100BD00081709070892B61F016950795F794E794D2
:100BE00080E090E0A0E0B0E8E82AF92A0A2B1B2B6D
:100BF00076956795579547952F5F3F4F77FDE7CFE0
:100C00000CC0440F551F661F771F17FD4160EE0C87
:100C1000FF1C001F111F21503040403090E0590749
:100C200090E0690790E4790760F32B8F3C8FDB013C
:100C3000CA018F779070A070B07080349105A105C3
:100C4000B10561F447FD0AC0E114F1040105110585
:100C500029F0405C5F4F6F4F7F4F40781A8EFE1730
:100C600011F081E08A8F4D8F5E8F6F8F78A383E0C4
:100C7000898FCE0149960E949506A096E2E10C94D8
:100C80006208ACE0B0E0E7E4F6E00C945608698353
:100C90007A838B839C83CE010196BE016B5F7F4F6D
:100CA0000E946A078D81823061F1823050F1843078
:100CB00021F48E81882351F12EC02F81388537FD94
:100CC00020C06E812F3131051CF06623F9F023C05E
:100CD0008EE190E0821B930B29853A854B855C85DC
:100CE00004C056954795379527958A95D2F7662380
:100CF000B1F050954095309521953F4F4F4F5F4F44
:100D00000EC020E030E040E050E009C02FEF3FEFA0
:100D10004FEF5FE704C020E030E040E050E8B90169
:100D2000CA012C96E2E00C947208DF92EF92FF92D7
:100D30000F931F93FC01E480F58006811781D18019
:100D40008081823048F480E090E0A0E1B0E0E82AC1
:100D5000F92A0A2B1B2BA5C0843009F49FC08230CE
:100D600021F4EE24FF24870105C0E114F1040105FC
:100D7000110519F4E0E0F0E096C0628173819FEF05
:100D8000623879070CF05BC022E83FEF261B370B77
:100D90002A3131052CF020E030E040E050E02AC05C
:100DA000B801A701022E04C076956795579547951F
:100DB0000A94D2F781E090E0A0E0B0E004C0880F90
:100DC000991FAA1FBB1F2A95D2F70197A109B10944
:100DD0008E219F21A023B1230097A105B10521F009
:100DE00081E090E0A0E0B0E09A01AB01282B392B24
:100DF0004A2B5B2BDA01C9018F779070A070B0701D
:100E000080349105A105B10539F427FF09C0205CA4
:100E10003F4F4F4F5F4F04C0215C3F4F4F4F5F4FDD
:100E2000E0E0F0E02030A0E03A07A0E04A07A0E4CC
:100E30005A0710F0E1E0F0E079018A0127C060383C
:100E4000710564F5FB01E158FF4FD801C7018F77A9
:100E50009070A070B07080349105A105B10539F48F
:100E6000E7FE0DC080E490E0A0E0B0E004C08FE3B6
:100E700090E0A0E0B0E0E80EF91E0A1F1B1F17FF6C
:100E800005C016950795F794E794319687E0169577
:100E90000795F794E7948A95D1F705C0EE24FF24CF
:100EA0008701EFEFF0E06E2F679566276795902F2B
:100EB0009F77D794DD24D7948E2F8695492F462B84
:100EC000582F5D29B701CA011F910F91FF90EF9034
:100ED000DF900895FC01DB01408151812281622F66
:100EE0006F7770E0221F2227221F9381892F880F9E
:100EF000822B282F30E0991F9927991F11969C93D8
:100F0000119721153105A9F54115510561057105A7
:100F100011F482E037C082E89FEF13969C938E9382
:100F200012979A01AB0167E0220F331F441F551F30
:100F30006A95D1F783E08C930DC0220F331F441FB5
:100F4000551F12968D919C911397019713969C9320
:100F50008E931297203080E0380780E0480780E4C5
:100F6000580758F314962D933D934D935C93179720
:100F700008952F3F310579F441155105610571053B
:100F800019F484E08C93089564FF03C081E08C938E
:100F900012C01C9210C02F57304013963C932E93D2
:100FA000129783E08C9387E0440F551F661F771FCD
:100FB0008A95D1F7706414964D935D936D937C93ED
:100FC0001797089597FB092E07260AD077FD04D0BE
:100FD00049D006D000201AF4709561957F4F08958E
:100FE000F6F7909581959F4F0895A1E21A2EAA1BBE
:100FF000BB1BFD010DC0AA1FBB1FEE1FFF1FA217C9
:10100000B307E407F50720F0A21BB30BE40BF50BC5
:10101000661F771F881F991F1A9469F7609570954E
:10102000809590959B01AC01BD01CF01089597FB80
:10103000092E05260ED057FD04D0D7DF0AD0001C9C
:1010400038F450954095309521953F4F4F4F5F4F65
:101050000895F6F790958095709561957F4F8F4F25
:101060009F4F0895AA1BBB1B51E107C0AA1FBB1FBE
:10107000A617B70710F0A61BB70B881F991F5A9524
:10108000A9F780959095BC01CD0108952F923F92CC
:101090004F925F926F927F928F929F92AF92BF9288
:1010A000CF92DF92EF92FF920F931F93CF93DF9334
:1010B000CDB7DEB7CA1BDB0B0FB6F894DEBF0FBE91
:1010C000CDBF09942A88398848885F846E847D84DE
:1010D0008C849B84AA84B984C884DF80EE80FD80E0
:1010E0000C811B81AA81B981CE0FD11D0FB6F89456
:1010F000DEBF0FBECDBFED010895EE0FFF1F0590BF
:10110000F491E02D09949F9305D00F9007FCEE5FBA
:1011100028C0CEC03FD0E8F3E894E0E0BB279F575B
:10112000F0F02AED3FE049EC06C0EE0FBB0F661F62
:10113000771F881F28F0B23A62077307840728F0E8
:10114000B25A620B730B840BE3959A9572F7803851
:1011500030F49A95BB0F661F771F881FD2F790480F
:101160009BC0EF93E0FF06C0A2EA2AED3FE049EC06
:101170005FEB37D0BFD00F90039401FC9058E8E6A6
:10118000F0E099C057FD9058440F551F59F05F3F4C
:1011900071F04795880F97FB991F61F09F3F79F099
:1011A00087950895121613061406551FF2CF46951B
:1011B000F1DF08C0161617061806991FF1CF86959D
:1011C000710561050894089587D030F08CD020F027
:1011D00031F49F3F11F41EF46BC00EF4E095E7FB71
:1011E00053C0E92FCFDF80F3BA1762077307840774
:1011F000950718F071F49EF58EC00EF4E0950B2E55
:10120000BA2FA02D0B01B90190010C01CA01A00158
:101210001124FF27591B99F0593F50F4503E68F1B3
:101220001A16F040A22F232F342F4427585FF3CFF4
:10123000469537952795A795F0405395C9F77EF4C5
:101240001F16BA0B620B730B840BBAF09150A1F00E
:10125000FF0FBB1F661F771F881FC2F70EC0BA0F94
:10126000621F731F841F48F4879577956795B7951C
:10127000F7959E3F08F0B3CF9395880F08F0992714
:10128000EE0F97958795089597F99F6780E870E02E
:1012900060E008959F3F31F0915020F48795779555
:1012A0006795B795880F911D9695879597F908953D
:1012B0009FEF80EC08959F938F937F936F93FF939D
:1012C000EF939B01AC01E3DBEF91FF912BD02F91CA
:1012D0003F914F915F91DBCB00240A9416161706BD
:1012E00018060906089500240A9412161306140617
:1012F00005060895092E0394000C11F4882352F07A
:10130000BB0F40F4BF2B11F460FF04C06F5F7F4F31
:101310008F4F9F4F0895E894BB2766277727CB010F
:1013200097F90895DF93CF931F930F93FF92EF9256
:10133000DF927B018C01689405C0DA2EEF0121D089
:10134000FE01E894A5912591359145915591AEF313
:10135000EF0147DFFE019701A801DA9479F7DF90EA
:10136000EF90FF900F911F91CF91DF910895B4DF1F
:1013700028F0B9DF18F0952309F086CF99CF112412
:10138000CBCF00DFA0F3959FD1F3950F50E0551F11
:10139000629FF001729FBB27F00DB11D639FAA27CA
:1013A000F00DB11DAA1F649F6627B00DA11D661F19
:1013B000829F2227B00DA11D621F739FB00DA11D3A
:1013C000621F839FA00D611D221F749F3327A00DF4
:1013D000611D231F849F600D211D822F762F6A2F90
:1013E00011249F5750408AF0E1F088234AF0EE0F15
:1013F000FF1FBB1F661F771F881F91505040A9F722
:101400009E3F510570F040CF87CF5F3FECF3983E91
:10141000DCF3869577956795B795F795E7959F5F88
:10142000C1F7FE2B880F911D9695879597F9089522
:04143000F894FFCF5E
:1014340057656C636F6D6520746F20656C656374AC
:101444006963000000000045010000000000000086
:02145400000096
:00000001FF
